:030000000200916A
:03002B00020EE1E1
:10003B00020EE253D9BF79012200000080FB1200AF
:10004B003EB9000302008BE49010007835790180F3
:10005B0002F0A3D8FCD9FA901034AA82AB8390009B
:10006B00A078AD79018015E493A3AC82AD838A822D
:10007B008B83F0A3AA82AB838C828D83D8E9D9E7DB
:10008B00120A9512004475D0007581BF751000756A
:10009B001110020049506C656173652077616974BA
:1000AB002E2E2E3F00444F4E4521204453313038E5
:1000BB0035207375636365737366756C6C79206338
:1000CB006F6E66696775726564213F00596F7520A5
:1000DB0063616E207475726E20706F776572206F1E
:1000EB0066663F004552524F5221204453313038FF
:1000FB0035204E4F5420636F6E6669677572656469
:10010B00213F00506C65617320636865636B2068E9
:10011B006172647761726520636F6E6E656374697B
:10012B006F6E733F00616E6420747279206167613A
:10013B00696E3F00010000000001000000A1860174
:10014B0000C3E09608A3E09608A3E09608A3E09608
:10015B0022E026F608A3E036F608A3E036F608A35D
:10016B00E036F622E0F608A3E0F608A3E0F608A3D3
:10017B00E0F622E6F008A3E6F008A3E6F008A3E613
:10018B00F022251010AF08F510400215118008F56C
:10019B001040021511D2AF22C0D0251010AF08F5B8
:1001AB0010500205118008F51050020511D2AFD086
:1001BB00D0222510C582C0E0E51134FFC583C0E015
:1001CB00E510C3958224F9F8E4C5A88583118582CF
:1001DB0010C5A8E8CEF0A3E520F0A37808E608F058
:1001EB00A3DEFAEFF0A3E58124FBF8E608F0A3E623
:1001FB0008F0A30808E608F0A3E608F0A31581159C
:10020B0081D0E0FED0E0F815811581E8C0E0EEC0AA
:10021B00E022851183851082E0A3FEE0A3F5207810
:10022B0008E0A3F608DFFAE0A3FFE0A3C0E0E0A339
:10023B00C0E0E0A3C0E0E0A3C0E0E4C5A885821065
:10024B00858311C5A8D083D08222D083D082C5F0FC
:10025B00E493A3C5F0C395F0F5F0E493A3C395F035
:10026B004005E5F0048001E475F002A42582F582D7
:10027B00E5F03583F583E493A3C0E0E493C0E0227B
:10028B00D083D082CCC0E0E493A360061202B514F5
:10029B0070FAE493A360061202D41470FAD0E0FC57
:1002AB00E493A3C0E0E493C0E022C0E0E493A3D3C3
:1002BB009C5010E493A3C39C400AD0E0D0E0D0E064
:1002CB000202A8A3A3A3D0E022C0E0E493A36C7026
:1002DB0009D0E0D0E0D0E00202A8A3A3D0E0220036
:1002EB000000000000000000000000000000000003
:1002FB000000000000FF33FF33000000000000008F
:10030B0000070007000000000007000700000020A6
:10031B0001FE1FFE1F20012001FE1FFE1F200138C2
:10032B00063C0E6408FF3FFF3F84091C0F18071E95
:10033B0030331C1E07C00170001C1E0733011E1E2C
:10034B001FB331E120E120B3311E1F001B803100B0
:10035B0000000000000B0007000000000000000080
:10036B00000000F807FF3F07380000000000000006
:10037B000000000000000000000000000000000072
:10038B000000000000000000000000000000000062
:10039B000000000000000000000000000000000052
:1003AB000000000000000000000000000000000042
:1003BB000000000000000000000000000000000032
:1003CB0000000000000030003000000000000000C2
:1003DB0030003C000FC003F0003C000F000300FC9A
:1003EB000FFE1F0336812161201B30FE1FFC0F0403
:1003FB002004200620FF3FFF3F0020002000200CA0
:10040B00380E3C032601238121C3207E203C20068D
:10041B001803304120412041204120E330BE1F0012
:10042B000FE00FFC081F08833F803F000800083FC8
:10043B000C3F1C2130212021206130C11F810FE096
:10044B000FF81F5C3046204320C130811F010F0184
:10045B000001000100013C813FF1037F000F001CF4
:10046B000FBE1FE33041204120E330BE1F1C0F3C69
:10047B00207E20C32081308118830EFE07FC0100F3
:10048B000000000000000000000000000000000061
:10049B000000000000000000000000000000000051
:1004AB000000000000000000000000000000002021
:1004BB000120012001200120012001200120010049
:1004CB000000000000000000000000000000000021
:1004DB000000000000000000000000000000000011
:1004EB00000000000000000000000000000000FC05
:1004FB003FFE3F0301010101010301FE3FFC3FFFF2
:10050B003FFF3F412041204120E330BE1F1C0FFC29
:10051B000FFE1F03300120012003300E1C0C0CFFBB
:10052B003FFF3F0120012001200738FE1FF807FF86
:10053B003FFF3F412041204120412041200120FF2E
:10054B003FFF3F810081008100810081000100FCA1
:10055B000FFE1F03300120812083308E1F8C0FFF75
:10056B003FFF3F4000400040004000FF3FFF3F0186
:10057B002001200120FF3FFF3F012001200120002F
:10058B000C001C0030002000200030FF1FFF0FFF6D
:10059B003FFF3FC000E00138071C0E0F3C0330FF4C
:1005AB003FFF3F002000200020002000200020FF04
:1005BB003FFF3F7800C003C0037800FF3FFF3FFFC2
:1005CB003FFF3F1C007000C0010007FF3FFF3FFCD7
:1005DB000FFE1F0330012001200330FE1FFC0FFF15
:1005EB003FFF3F810081008100C3007E003C000083
:1005FB00000000000000000000000000000000FFF1
:10060B003FFF3F810081008101C31F7E3E3C203CA8
:10061B000C7E1C6330E120C12183318E1F0C0F0334
:10062B000003000300FF3FFF3F030003000300FF35
:10063B000FFF1F0030002000200030FF1FFF0F3F77
:10064B0000FF01C00F003C003CC00FFF013F00FF4B
:10065B0001FF3F003EC001C001003EFF3FFF010014
:10066B000000000000000000000000000000003F40
:10067B0000FF00C001803F803FC001FF003F000131
:10068B0038013E8127C121612039201F200720001E
:10069B00000000000000000000000000000000004F
:1006AB00000000000000000000000000000000003F
:1006BB00000000000000000000000000000000002F
:1006CB00000000000000000000000000000000001F
:1006DB00000000000000000000000000000000000F
:1006EB0000000000000000000000000000000000FF
:1006FB001E403F2021202120212011E03FC03FFF41
:10070B003FFF3F4010202020206030C01F800F8013
:10071B000FC01F6030202020202020603040108030
:10072B000FC01F6030202020204010FF3FFF3F8074
:10073B000FC01F6032202220226022C03380132082
:10074B00002000FE3FFF3F2100210023000200801C
:10075B0007C00F6018201020104008E03FE03FFC5E
:10076B003FFC3F4000200020006000C03F803F0066
:10077B000020202020E33FE33F002000200000006A
:10078B00000000000000000000000000000000FC62
:10079B003FFC3F00060007800DC018603020200092
:1007AB000001200120FF3FFF3F002000200000E060
:1007BB003FE03F6000C01FC01F6000E03FC03FE054
:1007CB003FE03F4000200020006000C03F803F80A2
:1007DB000FC01F6030202020206030C01F800FE032
:1007EB003FE03F400420082008600CC00780030056
:1007FB00000000000000000000000000000000E00E
:10080B003FE03FC00040006000600060004000C05F
:10081B0010E0312021202320262024603C401800AA
:10082B000020002000FE1FFE3F202020200000E0C3
:10083B001FE03F0020002000200010E03FE03FF0D1
:10084B0003F007001C00300030001CF007F003E041
:10085B0007E03F0038E007E0070038E03FE0070023
:10086B00000000000000000000000000000000E09D
:10087B0001E027002600380018000EE007E00120F9
:10088B00302038202C20262023A021E020602000BF
:10089B00000000000000000000000000000000004D
:1008AB000000000000FF3FFF3F00000000000000C1
:1008BB00000000000000000000000000000000002D
:1008CB00000000000000000000000000000000001D
:1008DB00000000000000000000000000000000000D
:1008EB0000000000000000000000000000000000FD
:1008FB0000000000000000000000000000000000ED
:10090B000102030405060708090A0B0C0D0E0F1054
:10091B001112131415161718191A1B1C1D1E1F2044
:10092B002122232425262728292A2B2C2D2E2F3034
:10093B003132333435363738393A3B3C3D3E3F4024
:10094B004142434445464748494A4B4C4D4E4F5014
:10095B005152535455565758595A5B5C5D5E5F0064
:10096B00000000000000000000000000000000007C
:10097B00000000000000000000000000000000006C
:10098B00000000000000000000000000000000005C
:10099B00000000000000000000000000000000004C
:1009AB00000000000000000000000000000000003C
:1009BB00000000000000000000000000000000002C
:1009CB00000000000000000000000000000000001C
:1009DB000000000000000000000000000000007498
:1009EB00F71201BD8908750900E50824EAF582E5CF
:1009FB00093408F583E493901002F0901002E0F8AC
:100A0B007900E875F008A4C8AAF075F000A42AFADA
:100A1B0075F008E9A42AF9901000E8F0A3E9F07F3B
:100A2B000202021D75A40D75A5E775A70175D40FFC
:100A3B0075D50775DF0175E10575E2422275B98041
:100A4B007A008002000AEAC3941440F843B9C0E567
:100A5B00B9E5B9A2E550FA75A90275B28322D28C19
:100A6B00438922E589438E0CE58E758CB075C18068
:100A7B0043E60122120A48120A2F120A69C283D2D4
:100A8B0082D280C292D291D2AF2253D9BF120A7FA7
:100A9B001210631210437AFF7BFF12124E7C347DCF
:100AAB00107A827B007972121344901003E0D2E427
:100ABB00F07458901004F08007901004E02401F0BB
:100ACB00901004E0C39460502F7437901006F09090
:100ADB001003E0D2E3F0901003E0D2E1F0120E36F7
:100AEB00901003E0A2E440D1901004E0901005F0C8
:100AFB00901007E0901019F0740090100BF0800725
:100B0B0090100BE02401F090100BE0C3940A40030B
:100B1B00020BFE120D137459901004F0120C00907E
:100B2B00102BE0541FF0901017E0541FF090102F73
:100B3B00E0540FF090101BE0540FF0740190100A6A
:100B4B00F0800790100AE02401F090100AE0C394A3
:100B5B0010504090100AE0640C600890100AE0649A
:100B6B000D7006740E90100AF090100AE0790024B4
:100B7B0020F582E93410F583E0FA90100AE0790051
:100B8B00240CF582E93410F583E06A60B6740090AA
:100B9B0010D3F09010D3E06401701C7C447D107A6C
:100BAB000A7B0079721213447C6B7D107A1E7B00DA
:100BBB00790F121344803C90100BE0C39407500341
:100BCB00020B0B9010D3E06003020B0B7C837D10A8
:100BDB007A327B0079721213447CA27D107A0A7BE5
:100BEB000079281213447CC47D107A0A7B00790F9C
:100BFB0012134480FEC082C0837401901006F090E3
:100C0B001003E0D2E3F0901003E0D2E1F0120E36C5
:100C1B00901004E0901020F0901006E0901021F05E
:100C2B00901007E0901022F0901008E0901023F045
:100C3B007402901006F0901003E0D2E3F0901003D2
:100C4B00E0D2E1F0120E36901006E0901024F090F6
:100C5B001007E0901025F0901008E0901026F0742B
:100C6B0008901006F0901003E0D2E3F0901003E030
:100C7B00D2E1F0120E36901006E0901027F0901093
:100C8B0007E0901028F0901008E0901029F0740EF7
:100C9B00901006F0901003E0D2E3F0901003E0C246
:100CAB00E1F0120E36901006E090102AF09010072B
:100CBB00E090102BF07437901006F0901003E0D2F8
:100CCB00E3F0901003E0C2E1F0120E36901006E054
:100CDB0090102CF0901007E090102DF0740D9010E8
:100CEB0006F0901003E0D2E3F0901003E0C2E1F0C5
:100CFB00120E36901006E090102EF0901007E09038
:100D0B00102FF0D083D08222C082C0837401901048
:100D1B0006F07400901007F07400901008F090101B
:100D2B0003E0C2E3F0901003E0D2E1F0120E369034
:100D3B001005E090100CF0901006E090100DF09064
:100D4B001007E090100EF0901008E090100FF07468
:100D5B0002901006F07418901007F07400901008B1
:100D6B00F0901003E0C2E3F0901003E0D2E1F01238
:100D7B000E36901006E0901010F0901007E09010D7
:100D8B0011F0901008E0901012F07408901006F01B
:100D9B0074C3901007F07400901008F0901003E0EB
:100DAB00C2E3F0901003E0D2E1F0120E3690100681
:100DBB00E0901013F0901007E0901014F0901008D2
:100DCB00E0901015F0740E901006F0901019E013CF
:100DDB001313541F901007F0901003E0C2E3F09030
:100DEB001003E0C2E1F0120E36901006E0901016E0
:100DFB00F0901007E0901017F0740D901006F0743F
:100E0B0009901007F0901003E0C2E3F0901003E09C
:100E1B00C2E1F0120E36901006E090101AF090100E
:100E2B0007E090101BF0D083D0822274F11201BD29
:100E3B0074FC12018D9010D4780812016F9010037E
:100E4B00E0D2E0F0C2AD901003E0A2E3501290109C
:100E5B0003E0D2E2F0901003E0C2E3F0D2C580646D
:100E6B00901003E0C2E2F0D2C58059851082851143
:100E7B0083780812017E851082851183C082C0831E
:100E8B009010D8780812016FD083D08278081201A5
:100E9B005C851082851183C082C0839010DC780C36
:100EAB0012016FD083D082780C12014C4016901037
:100EBB0003E0A2E4500E901003E0C2E0F0901003A8
:100ECB00E0D2E4F0901003E0A2E0409F7404120122
:100EDB00A37F0802021D32C0E0C0D0E8C0E0E9C029
:100EEB00E0C008C009C082C083C0F0A2C250030298
:100EFB00102585C00874F0550812028B000380D0B2
:100F0B000FC0310FE0140F2510901004E0C333F520
:100F1B00C253C2FE901003E0A2E3E492E045C2F597
:100F2B00C2C2C5021025A2C14003020FC490100318
:100F3B00E0C2E4F0901003E0A2E35003021025900E
:100F4B001003E0A2E1400E901009E06402700674F9
:100F5B0003901009F0901009E012025500032510C0
:100F6B00730F820FA40FB30F901009E02401F090C0
:100F7B001006E0F5C2804C901003E0A2E2500B90FB
:100F8B001003E0D2E3F0D2C5802D901009E02401CC
:100F9B00F0901007E0F5C2802A901009E02401F0D0
:100FAB00901008E0F5C28072901003E0C2E0F0747C
:100FBB0000901009F0D2C480617400901009F0D237
:100FCB00C4D2C58055901003E0C2E4F0901009E044
:100FDB0012025501012510E60F1010E5C290100703
:100FEB00F0901009E02401F0901003E0A2E1401111
:100FFB00C2C17400901009F0901003E0C2E0F080C1
:10100B0019D2C18015E5C2901008F0C2C1740090CE
:10101B001009F0901003E0C2E0F0C2C0D0F0D08312
:10102B00D082D009D008D0E0F9D0E0F8D0D0D0E011
:10103B003275A60075A0FF2275A6FF22D2917A0504
:10104B007B0012139FC2917A0A7B0012139FD291DD
:10105B007A327B0012139F22D296D282D292121036
:10106B00431210477A0279831211EC7A03798512B5
:10107B0011EC7A93798C1211EC7A0179911211ECB3
:10108B007A0079831211EC7AB0793E1211EC7A0363
:10109B00793F1211EC7A1079401211EC7A567941A2
:1010AB001211EC7A1379421211EC7A467943121130
:1010BB00EC7A2379441211EC7A7679451211EC7A99
:1010CB000079461211EC7A5E79471211EC7A4F795E
:1010DB00481211EC7A4079491211EC7A61791712A6
:1010EB0011EC7AF9792B1211EC7A0A7B0012139F0F
:1010FB007A14791B1211EC7A11791A1211EC7A0D00
:10110B00791C1211EC7A3D791F1211EC7A147B00C9
:10111B0012139F7A0A79191211EC7A1A7919121192
:10112B00EC7A287B0012139F7A1279191211EC7A40
:10113B00287B0012139F7A20791E1211EC7A647BA4
:10114B000012139F7A60793C1211EC7A40793D12B0
:10115B0011EC7A3879341211EC7A3879351211ECAA
:10116B007A3879241211EC7A287B0012139F7A3C7F
:10117B0079241211EC7A1C79161211EC7A0679018A
:10118B001211EC7A0079551211EC7A0079021211D6
:10119B00EC7A0079031211EC7A0079041211EC7AD3
:1011AB00EF79051211EC7A0079061211EC7A0079BD
:1011BB00071211EC7A0179081211EC7A8F79091266
:1011CB0011EC79221211D612103C22D283C29289D1
:1011DB00A0C280D280D292C2832289A0C280D28048
:1011EB0022D283C29289A0C280D280D2928AA0C21C
:1011FB0080D280C2832274F81201BDEAFEEBFFD2CB
:10120B0083EFF9E9F91211E5EEF91211E5C2837FCB
:10121B000102021D74F81201BD8908EAFEEBFF12F0
:10122B001043AA0879031211ECEFFBEBFA790612C3
:10123B0011ECEEFA79071211EC79221211D67F011B
:10124B0002021D74F71201BDEAFEEBFFD2961210DB
:10125B00437A007B00790012121F79221211D67586
:10126B0008F97509C0EEFAEFFB121201EEFAEFFB6B
:10127B00121201AA0874FF2AF508EA70E8AA097489
:10128B00FF2AF509EA70DE7F0202021D74F11201DA
:10129B00BD890B8A0E8B0FECF91209EA750C0080D5
:1012AB0002050CE50CC39408400302133F850C08A0
:1012BB00750900E508250EFAE509350FFBA90B1298
:1012CB00121F7E007F2079221211D6750A00801022
:1012DB007AFF7BFF121201EFC313FFEE13FE050A19
:1012EB00E50AC3940E50BA901000850C08750900DE
:1012FB00E02508F8A3E03509F9E875F002A4C8AABF
:10130B00F075F000A42AFA75F002E9A42AF9E82492
:10131B00EAF582E93402F583E4935EF8A3E4935F84
:10132B00F9740068700374006960A57A007BF81289
:10133B00120180A37F0802021D74F31201BD8908FC
:10134B008A0C8B0D8C0A8D0B7E007F008026EEF8AD
:10135B00EFF9E875F00AA4C8AAF075F000A42AFA10
:10136B0075F00AE9A42AF9E50C28FAE50D39FBA971
:10137B0008121297E50A2EF582E50B3FF583E0FA8A
:10138B00EE2401FEEF3400FFEAFC743F6A70BF7F6E
:05139B000602021D2204
:000091016E
:00000001FF
